:04000000F6EF14F013
:1000080000C016F001C015F0E1CF17F0E2CF18F0EC
:100018009DAA69D09EAA67D0AECF00F2ABA20FD03E
:10002800AB98AECF00F2AB88010E02012125006E1D
:10003800000E2221016E00C021F201C022F2ABA401
:100048000FD00201AB9EAB8E010E2125006E000E73
:100058002221016E00C021F201C022F2AECF00F2CF
:10006800020100510D0A07E02C51000802E12B5152
:100078007E0801E316D0010E0301346F000E356FC0
:100088009D9A680E02012B25E16E030E2C21E26E6B
:10009800E66A2BC24EF32CC24FF32B6B2C6B006B12
:1000A80022D02C51000802E12B517E0805E2020EF5
:1000B8000301346F000E356F680E02012B25E16EC7
:1000C800030E2C21E26E00C2E6FF2BC24EF32CC2B7
:1000D8004FF3010E2B25006E000E2C21016E00C07F
:1000E8002BF201C02CF2F2AA0CD0F2A40AD0020121
:1000F800664A672A010E1127000E122313231423C0
:10010800F2949DA01ED09EA01CD00201174B182B64
:100118000101A9510201185D04E10101A851020180
:10012800175D0AE39D90CD90176B186B010E156F44
:10013800000E166FCD909D900B0ECF6EDB0ECE6E1F
:100148009E9016C000F015C001F017C0E1FF18C05E
:04015800E2FF1100B1
:0E015C00ACB202D00000FCD720C4ADFF1200F0
:10016A00C7B409D01F0EC514016E0150000A03E17D
:0A017A00010E006E01D0006A1200B1
:10018400F250026EF29E0500FF6A0150FE6E0050AE
:08019400FD6E02BEF28E1200A6
:0C019C0000000000000000000000120045
:0C01A800240E0D6E0D2EFED7000012007C
:1001B4009E961AC4C9FFB0C01BF4B1C01CF4B2C0EF
:1001C4001DF4B3C01EF4C7A422D00001B051B11174
:1001D400B211B3111BE004011B511C111D111E119E
:1001E4000EE103C2E1FF04C2E2FF040EE66E01C2A7
:1001F40000F002C201F0C4DF010E006E3BD0010E1C
:1002040004011B5F000E1C5B1D5B1E5BDCD7B0C0D2
:100214001BF4B1C01CF4B2C01DF4B3C01EF49EB6EE
:1002240022D00001B051B111B211B3111BE004018D
:100234001B511C111D111E110EE103C2E1FF04C26A
:10024400E2FF040EE66E01C200F002C201F098DF84
:10025400010E006E0FD0010E04011B5F000E1C5B2B
:100264001D5B1E5BDCD7C5BC02D0006A03D0C5840D
:06027400020E006E1200F4
:10027A00800E04011B6F1A1F1B5316E01B511A151F
:10028A00016E0152010ED8A4000E006E00B002D019
:10029A008B9A01D08B8A7DDF7CDF8B8480DF8B9405
:0A02AA007EDF1B331B9FE8D7120014
:1002B400B0C01CF4B1C01DF4B2C01EF4B3C01FF42E
:1002C40004011A6B1B6B1B51120802E11A518E08B0
:1002D40008E349DF005201E004D004011A4B1B2B50
:1002E400F2D70401120E1B5D02E18F0E1A5D03E3C7
:1002F4007B0E006E26D0C580C5A022D00001B0516F
:10030400B111B211B3111BE004011C511D111E11D6
:100314001F110EE103C2E1FF04C2E2FF050EE66E07
:1003240001C200F002C201F02BDF010E006E09D001
:10033400010E04011C5F000E1D5B1E5B1F5BDCD7FE
:04034400006A120039
:10034800B0C01AF4B1C01BF4B2C01CF4B3C01DF4A1
:10035800C582C5A220D00001B051B111B211B311AC
:1003680019E004011A511B111C111D110CE103C2E3
:10037800E1FF04C2E2FF060EE66E01C200F002C20F
:1003880001F0FCDE08D0010E04011A5F000E1B5BB1
:080398001C5B1D5BDED71200A7
:1003A000000000000000000000000000000000004D
:1003B000000000000000000000000000000000003D
:1003C000000000000000000000000000000000002D
:1003D000000000000000000000000000000000001D
:0403E0000000120007
:0403E400C5841200BA
:1003E800B0C01CF4B1C01DF4B2C01EF4B3C01FF4F9
:1003F8009E96C5869EB620D00001B051B111B211AB
:10040800B31119E004011C511D111E111F110CE13B
:1004180003C2E1FF04C2E2FF030EE66E01C200F070
:1004280002C201F0ABDE08D0010E04011C5F000E11
:100438001D5B1E5B1F5BDED70401C9CF1BF41A517D
:10044800000A02E1C58A01D0C59A9E96C588B0C047
:100458001CF4B1C01DF4B2C01EF4B3C01FF49EB6A4
:1004680020D00001B051B111B211B31119E004014B
:100478001C511D111E111F110CE103C2E1FF04C222
:10048800E2FF030EE66E01C200F002C201F076DE62
:1004980008D0010E04011C5F000E1D5B1E5B1F5B74
:0804A800DED71BC400F01200B6
:1004B00004011151390806E3300E115D03E3010E0A
:0804C000006E01D0006A120079
:1004C8000B6A0A6A096A00500402F4CF09F0F3CFF4
:1004D80008F001500502F4CF0BF0F3CF0AF00050FA
:1004E8000502F3500926F4500A22E86A0B2201504B
:1004F8000402F3500926F4500A22E86A0B2208C0C5
:1005080000F009C001F00AC002F00BC003F01200AD
:100518000B6A0A6A096A086A0E6A033408360450C4
:10052800085E0550D8A0053C095E0650D8A0063CD8
:100538000A5E0750D8A0073C0B5EE86AD8A0010EF7
:100548000E5E0336070E0C6E0334083609360A367B
:100558000B360E36045003A012D0085E0550D8A002
:10056800053C095E0650D8A0063C0A5E0750D8A094
:10057800073C0B5EE86AD8A0010E0E5E11D0082673
:100588000550D8B0053C09260650D8B0063C0A26C6
:100598000750D8B0073C0B26E86AD8B0010E0E26E3
:1005A80003360C2ED1D70234083609360A360B36F4
:1005B8000E36045003A012D0085E0550D8A0053CA2
:1005C800095E0650D8A0063C0A5E0750D8A0073C32
:1005D8000B5EE86AD8A0010E0E5E11D00826055001
:1005E800D8B0053C09260650D8B0063C0A26075064
:1005F800D8B0073C0B26E86AD8B0010E0E260236A2
:10060800070E0C6E0234083609360A360B360E36DB
:10061800045002A012D0085E0550D8A0053C095E1F
:100628000650D8A0063C0A5E0750D8A0073C0B5ECF
:10063800E86AD8A0010E0E5E11D008260550D8B081
:10064800053C09260650D8B0063C0A260750D8B003
:10065800073C0B26E86AD8B0010E0E2602360C2E8F
:10066800D1D70134083609360A360B360E3604500F
:1006780002A012D0085E0550D8A0053C095E0650BD
:10068800D8A0063C0A5E0750D8A0073C0B5EE86A73
:10069800D8A0010E0E5E11D008260550D8B0053C32
:1006A80009260650D8B0063C0A260750D8B0073CA1
:1006B8000B26E86AD8B0010E0E260136070E0C6E1E
:1006C8000134083609360A360B360E36045001A0B6
:1006D80012D0085E0550D8A0053C095E0650D8A087
:1006E800063C0A5E0750D8A0073C0B5EE86AD8A013
:1006F800010E0E5E11D008260550D8B0053C09261B
:100708000650D8B0063C0A260750D8B0073C0B263E
:10071800E86AD8B0010E0E2601360C2ED1D7003467
:10072800083609360A360B360E36045001A012D0A8
:10073800085E0550D8A0053C095E0650D8A0063CC6
:100748000A5E0750D8A0073C0B5EE86AD8A0010EE5
:100758000E5E11D008260550D8B0053C0926065073
:10076800D8B0063C0A260750D8B0073C0B26E86AE2
:10077800D8B0010E0E260036070E0C6E003408366F
:1007880009360A360B360E36045000A012D0085E21
:100798000550D8A0053C095E0650D8A0063C0A5E64
:1007A8000750D8A0073C0B5EE86AD8A0010E0E5E81
:1007B80011D008260550D8B0053C09260650D8B0F7
:1007C800063C0A260750D8B0073C0B26E86AD8B082
:1007D800010E0E2600360C2ED1D700B00ED00450D4
:1007E80008260550D8B0053C09260650D8B0063C66
:0C07F8000A260750D8B0073C0B26120060
:100804000B1E0A1E091E081E082AD8B4092AD8B4C9
:080814000A2AD8B40B2A1200D5
:10081C000450085E0550D8A0053C095E0650D8A0CF
:10082C00063C0A5E0750D8A0073C0B5E0336070E49
:10083C000C6E0334083609360A360B36045003A006
:10084C000ED0085E0550D8A0053C095E0650D8A015
:10085C00063C0A5E0750D8A0073C0B5E0DD008265C
:10086C000550D8B0053C09260650D8B0063C0A26DF
:10087C000750D8B0073C0B2603360C2EDAD70234BF
:10088C00083609360A360B36045003A00ED0085E23
:10089C000550D8A0053C095E0650D8A0063C0A5E5F
:1008AC000750D8A0073C0B5E0DD008260550D8B0D9
:1008BC00053C09260650D8B0063C0A260750D8B08D
:1008CC00073C0B260236070E0C6E0234083609362E
:1008DC000A360B36045002A00ED0085E0550D8A084
:1008EC00053C095E0650D8A0063C0A5E0750D8A00D
:1008FC00073C0B5E0DD008260550D8B0053C0926E8
:10090C000650D8B0063C0A260750D8B0073C0B2638
:10091C0002360C2EDAD70134083609360A360B3675
:10092C00045002A00ED0085E0550D8A0053C095E0C
:10093C000650D8A0063C0A5E0750D8A0073C0B5EB8
:10094C000DD008260550D8B0053C09260650D8B065
:10095C00063C0A260750D8B0073C0B260136070E7A
:10096C000C6E0134083609360A360B36045001A0D9
:10097C000ED0085E0550D8A0053C095E0650D8A0E4
:10098C00063C0A5E0750D8A0073C0B5E0DD008262B
:10099C000550D8B0053C09260650D8B0063C0A26AE
:1009AC000750D8B0073C0B2601360C2EDAD7003492
:1009BC00083609360A360B36045001A00ED0085EF4
:1009CC000550D8A0053C095E0650D8A0063C0A5E2E
:1009DC000750D8A0073C0B5E0DD008260550D8B0A8
:1009EC00053C09260650D8B0063C0A260750D8B05C
:1009FC00073C0B260036070E0C6E00340836093601
:100A0C000A360B36045000A00ED0085E0550D8A054
:100A1C00053C095E0650D8A0063C0A5E0750D8A0DB
:100A2C00073C0B5E0DD008260550D8B0053C0926B6
:100A3C000650D8B0063C0A260750D8B0073C0B2607
:100A4C0000360C2EDAD700B00ED004500826055014
:100A5C00D8B0053C09260650D8B0063C0A260750EB
:080A6C00D8B0073C0B26120074
:100A74001FDCD00E04011A6FDAEC00F011C41AF472
:100A8400DAEC00F012C41AF4DAEC00F0A9DC12007B
:100A9400086A080E0C6E003408360450085ED8B09C
:0E0AA40002D00826D89000360C2EF5D712008E
:100AB2008B90530E0D6E0D2EFED711C41AF43DEC21
:100AC20001F012C41AF43DEC01F069DC11C41AF40D
:100AD2003DEC01F013C41AF43DEC01F060DC11C4EA
:100AE2001AF43DEC01F014C41AF43DEC01F057DCA9
:100AF20011C41AF43DEC01F015C41AF43DEC01F0F6
:100B02004EDC11C41AF43DEC01F016C41AF43DECAB
:100B120001F045DC11C41AF43DEC01F017C41AF4DB
:100B22003DEC01F03CDC11C41AF43DEC01F018C4B8
:100B32001AF43DEC01F033DC11C41AF43DEC01F07F
:100B420019C41AF43DEC01F02ADC8B80100E0D6EF4
:080B52000D2EFED70000120079
:100B5A005AEC01F0D00E04011A6FDAEC00F011C45D
:100B6A001AF4DAEC00F0A4EC01F0D10E04011A6FC9
:100B7A00DAEC00F004011A6B32DC00C012F42DDC4E
:060B8A0012C400F012008D
:100B900011C400F00032009E0032009E0032009E20
:100BA0000032009E12C4E1FF13C4E2FF300E0024A5
:100BB000E66E010E04011225E16E000E1321E26EB5
:100BC0000F0E1115006E300E002600C0E6FF020E5B
:0E0BD0001225E16E000E1321E26EE66A12009D
:100BDE000401116BBBDF800E00100301326F336B0B
:100BEE00000E3313000E336F0401116B32C312F477
:080BFE003ADF02012F6B120027
:100C060004010D6B0E6B000E0E5D02E10A0E0D5D0A
:100C16000BE20D510B25E16E0E510C21E26E200EFA
:100C2600E66E0D4B0E2BEFD70D510B25E16E0E51D7
:100C36000C21E26EE66A010E0D5F000E0E5B0D5191
:100C46000B250F6F0E510C21106F0A0E046E000E4D
:100C5600056E066E076E07C400F008C401F009C4ED
:100C660002F00AC403F055DC08C000F009C001F028
:100C76000AC002F00BC003F0300E00260FC4E1FFDD
:100C860010C4E2FF00C0E6FF0A0E046E000E056EF9
:100C9600066E076E07C400F008C401F009C402F02E
:100CA6000AC403F036DC00C007F401C008F402C031
:100CB60009F403C00AF4000E046E031808E1045098
:100CC600021805E10450011802E10050000A01E192
:0E0CD60005D0010E0D5F000E0E5BB1D71200AF
:100CE4000401116B38DF00C02DF2010E0401116FF5
:100CF40032DF00C02EF2020E0401116F2CDF00C09F
:100D0400EAF3030E0401116F26DF00C0E9F3040EB9
:100D14000401116F20DF00C0E8F3050E0401116F18
:100D24001ADF00C0ECF3060E0401116F14DF00C0DB
:100D3400EBF3EAC311F4440E0401126F030E136FB4
:100D440025DF3A0E0301466F2EC211F4470E04014B
:100D5400126F030E136F1ADF3A0E0301496F2DC28F
:100D640011F44A0E0401126F030E136F0FDF030117
:100D74004C6BE8C311F4360E0401126F030E136FAB
:100D840005DF2D0E0301386FECC311F4390E040195
:100D9400126F030E136FFADE2D0E03013B6FEBC3CC
:100DA40011F43C0E0401126F030E136FEFDE030106
:040DB4003E6B120080
:100DB800086A096A100E0C6E0134083609360450A8
:100DC800085E0550D8A0053C095ED8B007D004508D
:100DD80008260550D8B0053C0926D89000360136BB
:060DE8000C2EEAD71200F8
:100DEE000401096B0A6B07C403F008C404F007C4BE
:100DFE0005F008C406F003C0E9FF04C0EAFFEE5098
:100E0E00200A04E109510A1101E110D0010E096F07
:100E1E00000E0A6F03C0E9FF04C0EAFF05C0E1FF40
:100E2E0006C0E2FFEECFE6FF054A062A03C001F038
:100E3E0004C002F0034A042A01C0E9FF02C0EAFF1F
:100E4E00EE50000AD8E107C400F008C401F0120009
:100E5E00040E0C6E3A0E0D6E0D2EFED70C2EFCD718
:040E6E00000012006E
:100E7200030E006E07C40EF4000E04010F6F005043
:100E820005E00E370E910F37FF0FFAD7106B3C0EAD
:100E92000725F66E460EF76E000EF722000EF86E6C
:100EA200000EF8220900F5CF30F20C6B0D6B000E2C
:100EB2000D5D02E1080E0C5DD8B0D0D0400E0A6F75
:100EC200000E0B6F000E006E0B51005C02E10A5126
:100ED200000819E2300E0A25E16E020E0B21E26EC5
:100EE200010E0A5D006E000E0B59016E300E0024D9
:100EF200E96E020E0120EA6EEECFE6FF010E0A5FF6
:100F0200000E0B5BDFD70E510C25006E0F510D2129
:100F1200016E3C0E0024F66E460E0120F76E000EA6
:100F2200F86E000EF8220900F5CF30F2106B080EB1
:100F32000A6F000E0B6F000E006E0B51005C02E197
:100F42000A51000875E20AC411F4300EE96E020E6D
:100F5200EA6E1051E926D8B0EA2AEECF12F4080E52
:100F62001025006E016A000E0122300E0024E96E87
:100F7200020E0120EA6EEECF13F4100E1025006E61
:100F8200016A000E0122300E0024E96E020E0120D9
:100F9200EA6EEECF14F4180E1025006E016A000EF0
:100FA2000122300E0024E96E020E0120EA6EEECF1D
:100FB20015F4200E1025006E016A000E0122300E7B
:100FC2000024E96E020E0120EA6EEECF16F4280E1E
:100FD2001025006E016A000E0122300E0024E96E17
:100FE200020E0120EA6EEECF17F4300E1025006ECD
:100FF200016A000E0122300E0024E96E020E012069
:10100200EA6EEECF18F4380E1025006E016A000E5B
:101012000122300E0024E96E020E0120EA6EEECFAC
:1010220019F446DD102B010E0A5F000E0B5B83D70D
:101032000A6B0B6B09510B5D02E108510A5D0BE271
:10104200070E0C6E7D0E0D6E0D2EFED70C2EFCD7EC
:0E1052000A4B0B2BEFD70C4B0D2B29D712009E
:10106000A69C07C4A9FFA69EA680A8CF00F01200E8
:1010700007C4E9FF08C4EAFFEE500401091905E1BD
:1010800007C400F008C401F010D007C400F008C481
:1010900001F0074B082B00C0E9FF01C0EAFFEECFCB
:0C10A00000F00052E5E1006A016A120055
:1010AC000D0E0401206FAEEC00F00A0E0401206F4F
:0610BC00AEEC00F0120092
:1010C2000401086B075109081BE20A0E046E07C4EB
:1010D20000F0DFDC00C008F400C008F40837089113
:1010E2000837089108370891083708910A0E046EEC
:1010F20007C400F0CEDC08C000F00050081302D094
:0A11020007C408F408C400F012004E
:10110C0007C4E9FF08C4EAFFEECF09F4000E04019E
:10111C000A6F000E0A6F000E0A1902E1200E09195F
:10112C0007E0000E0A1902E1090E091901E003D0CB
:10113C00074B082BE5D70B6B0C6B0D6B0E6B000E76
:10114C000A1902E12D0E091905E10D4B0E2B074B67
:10115C00082B08D0000E0A1902E12B0E091902E126
:10116C00074B082B07C4E9FF08C4EAFFEECF09F4CC
:10117C00000E0A6F000E0A6F09C411F458EC02F04D
:10118C00005219E00BC400F00CC401F00A0E046EFE
:10119C00000E056E64EC02F0300E095D026E000E5E
:1011AC000A59036E025000240B6F035001200C6F80
:1011BC00074B082BD7D70D510E1108E00B51000827
:1011CC00006E0CC401F0000E015604D00BC400F0EC
:0611DC000CC401F012003A
:1011E20004010A6B07C4E9FF08C4EAFFEECF09F461
:1011F2000951000A0FE009C420F4AEEC00F004012A
:101202000A2B0A510725E96E000E0821EA6EEECF7D
:0612120009F4EED7120002
:101218000BC400F004010B07005228E007C4E9FFE3
:1012280008C4EAFFEE50000A0CE007C4E9FF08C44E
:10123800EAFF09C4D9FF0AC4DAFFEE50DE1801E15B
:101248000FD007C4E9FF08C4EAFF09C4D9FF0AC4DC
:10125800DAFFDE50EE5C006E016A000E015A08D01B
:101268000401074B082B094B0A2BD2D7006A016AE5
:02127800120062
:10127A0002012F5301E015D00401116B69DC7F0EC6
:10128A0000140301326F336B000E3317000E336FF5
:10129A000401116B32C312F43AEC05F0010E02019B
:0412AA002F6F120090
:1012AE0007C4F6FF08C4F7FF09C4F8FF0900F5CF1D
:1012BE0000F0005212E007C4F6FF08C4F7FF09C49D
:1012CE00F8FF0900F5CF20F4AEEC00F0010E04019A
:0C12DE000727000E08230923E3D71200A5
:1012EA0007C402F008C403F002C000F003C001F012
:1012FA00024A032A00C0E9FF01C0EAFFEE5201E0F8
:10130A00F3D704010751025C006E08510358016EBD
:0A131A00010E005E000E015A1200E1
:10132400220E0C6E086A096A0A6A0B6A0C06D8B4A3
:101334001FD0D8900B320A320932083203320232FB
:1013440001320032D8A0F2D70C06D8B409D0045028
:1013540008260550092206500A2207500B22EAD714
:10136400045008260550092206500A2207500B2271
:02137400120065
:101376000401076B086B800E0819006E800E005C76
:1013860002E1080E075D10E20751010F116F126BA3
:10139600136B146B156B166B176B186B196B59EC7B
:0A13A60005F0074B082BE7D71200F3
:1013B0000450000A12E10550000A0FE10650000A2D
:1013C0000CE10750000A09E1FF0E006EFF0E016EEE
:1013D000FF0E026E7F0E036E99D00C6A07BE0C2AB8
:1013E0000D6A0B6A0A6A096A086A03500210011042
:1013F0000010D8B485D0035007180E6E0EBE0D1E17
:1014000007AE0BD0041E051E061E071E042AD8B404
:10141000052AD8B4062AD8B4072A03AE0BD0001E7A
:10142000011E021E031E002AD8B4012AD8B4022AC3
:10143000D8B4032A035007100E6E0EBE1DD00EEC5A
:1014400004F00CBE36D00DAE5BD0001E011E021E95
:10145000031E002AD8B4012AD8B4022AD8B4032A19
:10146000081E091E0A1E0B1E082AD8B4092AD8B461
:101470000A2AD8B40B2A44D007AE15D003BE0DD02B
:1014800003500B6E02500A6E0150096E0050086E38
:10149000036A026A016A006AD6D7036A026A016AAD
:1014A000006A002A000C031E021E011E001E0C8E84
:1014B000C6D7082AD8B4092AD8B40A2AD8B40B2A1D
:1014C0000450085CD8A4BFD70550095CD8A4BBD78A
:1014D00006500A5CD8A4B7D707500B5CD8A4B3D782
:1014E0000B6A0A6A096A086A002AD8B4012AD8B4C1
:1014F000022AD8B4032A03AEA6D70E6A0E88FF0CC0
:0E1500000E6A0CA002D002EC04F0000F1200E4
:0A150E00530E0D6E0D2EFED71200D5
:0E151800810E0D6E0D2EFED700000000120099
:101526000134083609360450085E0550D8A0053C3B
:10153600095E003601360F0E0C6E01340836093688
:10154600045000A006D0085E0550D8A0053C095EF0
:1015560005D008260550D8B0053C092600360136C8
:101566000C2EEBD700B006D0045008260550D8B094
:08157600053C092600001200EB
:10157E00F1C300F00032009E0032009E0032009E49
:10158E000032009EC50E0024F66E530EF76E000E4E
:10159E00F722000EF86E000EF8220900F5CF00F0CB
:1015AE00F2C3E1FFF3C3E2FF00C0E6FF010E030149
:1015BE00F225E16E000EF321E26E0F0EF115006EB4
:1015CE00C50E0024F66E530EF76E000EF722000EB7
:1015DE00F86E000EF8220900F5CF00F000C0E6FF0D
:1015EE00020EF225E16E000EF321E26EE66A1200A3
:1015FE00F3C301F0010E006E015004E000360090BE
:10160E00FF0FFBD700C0F7F3001C0301F66FF56B5D
:10161E00F1C3E9FFF2C3EAFFF46BF451070822E3CA
:10162E00F651EF16120EE926F651EF16CEEC00F03B
:10163E00F751EF12CEEC00F0120EE95EF751EF14F7
:10164E00006E0CE0F4C301F0010E006E015004E0D8
:10165E0000360090FF0FFBD70050F51351DF50DF1F
:0A166E00F42BDBD7F5C300F01200E7
:10167800F3C301F0010E006E015004E00036009043
:10168800FF0FFBD700C0F7F3001E00C0F6F3F1C34D
:10169800E9FFF2C3EAFF0050EF16120EE926030134
:1016A800F56BF551070815E3F5C300F0F4C301F035
:1016B800005004E00132019EFF0FFBD7F651EF16F0
:1016C80001A002D0F751EF1223DFF751EF12F52BEB
:0C16D800E8D7120EE95E17DF16DF1200E3
:1016E400F3C301F0010E006E015004E000360090D7
:1016F400FF0FFBD700C0F5F3001EF1C3E9FFF2C3EF
:10170400EAFF0050EF16120EE9260050EF162FECF8
:1017140007F00301F551EF12120EE95EFBDEF551FD
:10172400EF14F46FF451000A000ED8A4010EF46F04
:0A1734002FEC07F0F4C300F01200E0
:10173E000301F56B050EF55D0AE2F551F325E16E39
:10174E00000EF421E26E200EE66EF52BF3D7F55166
:10175E00F325E16E000EF421E26EE66AF507F5510F
:10176E00F325F66F000EF421F76F0A0E046E000ECD
:10177E00056EF1C300F0F2C301F0DCEC06F008C018
:10178E0000F009C001F0300E0026F6C3E1FFF7C3EA
:10179E00E2FF00C0E6FF0A0E046E000E056EF1C3F6
:1017AE0000F0F2C301F0DCEC06F000C0F1F301C072
:1017BE00F2F3000E011802E1000E001801E102D052
:0617CE00F507CDD7120063
:1017D400030E0B6E8A0E0C6E550E0D6E0D2EFED77B
:0E17E4000C2EFCD70B2EFAD7000000001200CE
:1017F200F3C304F0F4C305F0F1C302F0F2C303F043
:10180200F5C300F0F6C301F0010E0301F55F000E0F
:10181200F65B005001100FE004C0E9FF05C0EAFFCB
:1018220002C0E1FF03C0E2FFEECFE6FF024A032A55
:10183200044A052AE5D7F1C300F0F2C301F0120011
:10184200F1C3F5F3F2C3F6F3F5C307F408DC00C005
:10185200F7F3000E0301F86F000EF81902E1000E13
:10186200F71901E12DD0800E006E800EF619005C92
:1018720002E1F551FE0801E223D0F7C320F4AEECF9
:1018820000F00301F151F55D006EF251F659016E5F
:101892000050F325E16E0150F421E26EF7C3E6FF3A
:1018A200A30E0C6E550E0D6E0D2EFED70C2EFCD710
:1018B200F54BF62B000EF81902E1000EF719C4E100
:0218C200120012
:1018C4000900F5CFE6FF0006FBE10106F9E112008D
:1018D400020E0C6E9E0E0D6E0D2EFED70C2EFCD736
:0418E40000001200EE
:1018E800130E806E070EC16E0F0E926E9298898845
:1018F80092869280FF0E816EFF0E936E9382826AAB
:10190800FF0E946E948E949C94909482949A9494DE
:10191800D0EC01F08B80D0EC01F08B9AD0EC01F088
:081928008B94D0EC01F01200D9
:10193000F3C3F6FFF4C3F7FFF5C3F8FF0900F5CFD3
:1019400000F0005218E0F3C3F6FFF4C3F7FFF5C34D
:10195000F8FF0900F5CF00F0F1C3E1FFF2C3E2FFA9
:1019600000C0E6FF0301F14BF22B010EF327000E3E
:10197000F423F523DDD7F1C3E1FFF2C3E2FFE66A0A
:02198000120053
:101982005C0E02010D6F010E0E6F200E0F6F040E22
:10199200106FFF0E1D6FFF0E1E6F000E1F6F000EE9
:1019A200206FFF0E196FFF0E1A6F000E1B6F000ED5
:1019B2001C6FFF0E236FFF0E246F000E256F000EAB
:1019C200266FAC8A900EAB6E948E949C9EAA03D026
:0819D200AECF00F0FBD71200BC
:0E19DA009482949A949482928B9A8B94120029
:1019E8000301F2AF0BD0F3C3E1FFF4C3E2FF2D0E06
:1019F800E66EF11FF21FF14BF22B06D0F3C3E1FFA5
:101A0800F4C3E2FF200EE66EF1C300F0F2C301F06A
:101A180001320032019E01320032019E0132003251
:101A2800019E01320032019E00C0F5F3010EF3253C
:101A3800F86F000EF421F96F0A0E046E4AEC05F0F7
:101A48000A0E046E4AEC05F008C000F0300E0026BD
:101A5800F8C3E1FFF9C3E2FF00C0E6FF010EF3257A
:101A6800E96E000EF421EA6EEE50300A08E1010E2C
:101A7800F325E16E000EF421E26E200EE66E020EF2
:101A8800F325F86F000EF421F96F0A0E046EF5C302
:101A980000F04AEC05F008C000F0300E0026F8C34C
:101AA800E1FFF9C3E2FF00C0E6FFF1C3F6F3F2C3BA
:101AB800F7F30F0EF115006EF2C301F0000E0116D8
:101AC80000C0F6F301C0F7F3710E046E020E056E46
:101AD80064EC02F000C0F6F301C0F7F3030EF3253F
:101AE800E16E000EF421E26E2E0EE66E040EF32572
:101AF800F86F000EF421F96FE80E046E030E056E00
:101B0800F6C300F0F7C301F0DCEC06F0300E002657
:101B1800F8C3E1FFF9C3E2FF00C0E6FF050EF325B5
:101B2800F86F000EF421F96F640E046E000E056E56
:101B3800F6C300F0F7C301F0DCEC06F00A0E046E01
:101B4800000E056EDCEC06F008C000F009C001F0DC
:101B5800300E0026F8C3E1FFF9C3E2FF00C0E6FF3C
:101B6800060EF325E16E000EF421E26EE66A070E1A
:101B7800F325E16E000EF421E26EE66A080EF32505
:101B8800E16E000EF421E26EE66A010EF32504010F
:101B9800076F000E0301F4210401086FF7EC06F04B
:101BA800F5C300F0000E016EE80E046E030E056E1C
:101BB80064EC02F00301F65100240001D16F030127
:101BC800F75101200001D26F000ED36FD46F1200BD
:101BD800000E0301F21902E1000EF1193AE0F1C317
:101BE800E9FFF2C3EAFFEE5234E0F3C307F4F4C3AB
:101BF80008F475EC09F000C00BF4F1C307F4F2C364
:101C080008F4F3C309F4F4C30AF40CEC09F0000E69
:101C1800011802E1000E001805E1F1C300F0F2C35B
:101C280001F019D0010E0301F1250401076F000E20
:101C38000301F2210401086FF3C3E9FFF4C3EAFFCB
:101C4800EECF09F438EC08F000C0F1F301C0F2F36C
:081C5800BFD7006A016A120007
:101C6000F1C304F0F2C305F004C0E9FF05C0EAFFC8
:101C7000EE5203E0044A052AF7D704C002F005C07B
:101C800003F0044A052AF3C300F0F4C301F0030192
:101C9000F34BF42B00C0E9FF01C0EAFF02C0E1FFF3
:101CA00003C0E2FFEECFE6FF02C0E9FF03C0EAFF98
:101CB000EE5201E0E2D7F1C300F0F2C301F01200EE
:101CC000F1C304F0F2C305F004C002F005C003F054
:101CD000044A052AF3C300F0F4C301F00301F34BF7
:101CE000F42B00C0E9FF01C0EAFF02C0E1FF03C01E
:101CF000E2FFEECFE6FF02C0E9FF03C0EAFFEE52CB
:0E1D000001E0E2D7F1C300F0F2C301F01200DF
:101D0E000450000A08E10550000A05E1FF0E006EBE
:101D1E007F0E016E58D00D6A096A086A01500010D4
:101D2E00D8B4000C015005180A6E0ABE0D1E0B6ABF
:101D3E0005AE05D0041E051E042AD8B4052A01AE30
:101D4E0005D0001E011E002AD8B4012A015005102C
:101D5E000A6E0ABE10D093EC0AF00BB020D00DAE76
:101D6E00000C001E011E002AD8B4012A081E091EEE
:101D7E00082AD8B4092A000C05AE0DD001BE07D032
:101D8E000150096E0050086E016A006AE8D7016AB8
:101D9E00006A002A000C011E001E0B2ADDD7082A3D
:101DAE00D8B4092A0450085CD8A4D9D70550095CC8
:101DBE00D8A4D5D7096A086A002AD8B4012A01AE78
:081DCE00CED70000FF0C12004B
:101DD6000301F56BF66BF351F5250401076F30EC43
:101DE60008F000C0F7F3000E0301F86F000EF819B3
:101DF60002E1000EF71901E122D0800E006E800E7E
:101E0600F619005C02E1F5511F0801E218D0F55100
:101E1600F125E16EF651F221E26EF7C3E6FF070EF9
:101E26000C6E7D0E0D6E0D2EFED70C2EFCD7F54BCF
:101E3600F62B000EF81902E1000EF719CCE1F55168
:101E4600F125006EF651F221016E010E005CE16E85
:0A1E5600000E0158E26EE66A120069
:101E6000020E0301F16F000EF26F56EC08F0030151
:101E7000F56BF66B9D9A680E4E25E16E030E4F21B1
:101E8000E26EE66A800E4F19006E800E005C02E181
:101E9000160E4E5DD8B0FBD0800E006E800E4F192E
:101EA000005C02E14E511308D8B0F1D0020EF36F7E
:101EB000000EF46F800EF419006E800E4F19005C56
:101EC00002E14E51F35D43E2680EF325E96E030E25
:101ED000F421EA6EEECF01F001503B0A35E1680EC5
:101EE000F325E16E030EF421E26EE66A500EF5254D
:101EF000F96F030EF621FA6F680EF1250401076FE2
:101F0000030E0301F2210401086F86EC08F0F9C307
:101F1000E1FFFAC3E2FF00C0E6FF680E0301F1250E
:101F20000401076F030E0301F2210401086FF1ECB5
:101F300008F056EC08F00301F54BF62B010EF325E3
:101F4000F16F000EF421F26FF34BF42BB3D7500E68
:101F5000F525F96F030EF621FA6F680EF1250401DD
:101F6000076F030E0301F2210401086F86EC08F0ED
:101F7000F9C3E1FFFAC3E2FF00C0E6FF55C3F7F380
:101F8000000E0301F86F54C355F353C354F3F7C362
:101F900053F350C3E8F351C3ECF352C3EBF3F7C36D
:101FA000E9F3F75106080AE2E96B0D0E0401076F29
:101FB000520E086F000E096F57EC09F054C3EAF394
:101FC00055C32EF202012D6BEFEC05F00401116BED
:101FD000126B3AEC05F02EC207F461EC08F000C079
:101FE00012F4010E116F3AEC05F0EAC307F461EC4C
:101FF00008F000C012F4020E116F3AEC05F0E9C3CC
:1020000007F461EC08F000C012F4030E116F3AEC13
:1020100005F0E8C307F461EC08F000C012F4040E08
:10202000116F3AEC05F0ECC307F461EC08F000C066
:1020300012F4050E116F3AEC05F0EBC307F461ECF6
:1020400008F000C012F4060E116F3AEC05F0070E0E
:102050000401116F100E126F3AEC05F08D0E0401A1
:10206000076F520E086F000E096F57EC09F056EC1F
:1020700008F05D0E0401076F530E086F000E096F24
:1020800057EC09F03DEC09F072EC06F012D0700E3E
:102090000401076F4F0E086F000E096F57EC09F02F
:1020A000450E0401076F4E0E086F000E096F57ECC6
:0420B00009F0120021
:1020B400A6A202D00000FCD7A69CF1C3A9FFF2C3DC
:1020C400A8FFA69EA684F2CF00F0F29E550EA76E3E
:1020D400AA0EA76EA68200BE02D0F29E01D0F28E96
:0E20E400A694A1B802D00000FCD7A19812006B
:1020F200F2C300F00032009E0032009E0032009EC9
:102102000032009EC50E0024F66E530EF76E000ECE
:10211200F722000EF86E000EF8220900F5CF00F04B
:10212200F3C3E1FFF4C3E2FF00C0E6FF010E0301C7
:10213200F325E16E000EF421E26E0F0EF215006E31
:10214200C50E0024F66E530EF76E000EF722000E37
:10215200F86E000EF8220900F5CF00F000C0E6FF8D
:10216200020EF325E16E000EF421E26EF1C300F0DF
:102172000032009E0032009E0032009E0032009E1D
:10218200C50E0024F66E530EF76E000EF722000EF7
:10219200F86E000EF8220900F5CF00F000C0E6FF4D
:1021A200030EF325E16E000EF421E26E0F0EF1151F
:1021B200006EC50E0024F66E530EF76E000EF72267
:1021C200000EF86E000EF8220900F5CF00F000C0F4
:1021D200E6FF040EF325E16E000EF421E26EE66ADC
:0221E2001200E9
:1021E400F1C3F6FFF2C3F7FFF3C3F8FF0900F5CF1D
:1021F40001F00150000816E2F1C3F6FFF2C3F7FF45
:10220400F3C3F8FF0900F5CF07F4F4C308F4F5C3EA
:1022140009F439EC07F0010E0301F127000EF22353
:06222400F323DED71200D7
:10222A000301F46B030EF45D0AE2F451F225E16E48
:10223A00000EF321E26E200EE66EF42BF3D7F45172
:10224A00F225E16E000EF321E26EE66AF407F4511C
:10225A00F225F56F000EF321F66F0A0E046EF1C334
:10226A0000F04AEC05F008C000F0300E0026F5C375
:10227A00E1FFF6C3E2FF00C0E6FF0A0E046EF1C3F7
:10228A0000F04AEC05F000C0F1F30050000A01E149
:08229A0002D0F407DCD71200AA
:1022A2008B900D0E0C6EFB0E0D6E0D2EFED70C2EAE
:1022B200FCD700000000090E0401116F126B136BB2
:1022C200146B156B166B176B186B196B59EC05F0C9
:1022D2000A0E116F010E126F010E136F010E146FB1
:1022E200010E156F010E166F010E176F010E186F9A
:1022F200010E196F59EC05F00B0E116F070E126FDC
:10230200070E136F070E146F070E156F070E166F69
:10231200070E176F070E186F070E196F59EC05F0AD
:102322000C0E116F010E126F010E136F010E146F5E
:10233200010E156F010E166F010E176F010E186F49
:10234200010E196F59EC05F00F0E116F126B136B22
:10235200146B156B166B176B186B196B59EC05F038
:10236200410E0C6EEE0E0D6E0D2EFED70C2EFCD70E
:102372000000BBEC09F08B80030E0B6E8A0E0C6E14
:10238200550E0D6E0D2EFED70C2EFCD70B2EFAD746
:0623920000000000120033
:102398006A0E0101FC6F010EFD6F000EFE6F000E4C
:1023A800FF6FB40E0201096F020E0A6F000E0B6F69
:1023B800000E0C6F480E056F030E066F000E076FB8
:1023C800000E086FE80E0101F46F030EF56F1A0E88
:1023D800F66F040EF76FB40EF06F010EF16F1A0E60
:1023E800F26F040EF36FE40EF86F030EF96F000E30
:1023F800FA6F000EFB6F949894968B988B9694883E
:0C2408009486C79EC79C380EC66E12005A
:10241400F1C300F00032009E0032009E0032009EA4
:102424000032009E0A0E0002F3CF01F00F0E0301EA
:0A243400F115006E015000261200A1
:10243E000301F96BFA6BF1C3FBF3F2C3FCF3F3C3C5
:10244E00FDF3F4C3FEF3800EF419006E800E005CF3
:10245E0008E1000EF35D05E1000EF25D02E1000EF3
:10246E00F15D10E2010EF96F000EFA6FFB6BFC6B63
:10247E00FD6BFE6BF151FB5FF251FC5BF351FD5BAB
:10248E00F451FE5BFBC307F4FCC308F4FDC309F46F
:10249E00FEC30AF4F5C30BF4F6C30CF403EC06F01A
:1024AE000B0E0301F76F000EF86F000E006EF85161
:1024BE00005C02E1F751000819E2F751F525E16ED3
:1024CE00F851F621E26E010EF75D006E000EF8591E
:1024DE00016E0050F525E96E0150F621EA6EEECF41
:1024EE00E6FF010EF75F000EF85BDFD7F5C3E1FFE5
:1024FE00F6C3E2FF200EE66EF951FA111AE0F76B01
:10250E00F86BF751F525E96EF851F621EA6EEE50AB
:10251E00200A03E1F74BF82BF4D7010EF75F000EFC
:10252E00F85BF751F525E16EF851F621E26E2D0EAE
:04253E00E66E120033
:10254200F1C3E9FFF2C3EAFFEE50000810E2F1C363
:10255200E9FFF2C3EAFFEECF07F4F3C308F4F4C3D2
:1025620009F439EC07F00301F14BF22BE9D7120021
:10257200060E0301F125E96E000EF221EA6EC00E8D
:10258200EE24F36F120EEE20F46F000EF56FF66F6D
:10259200F3C300F0F4C301F0F5C302F0F6C303F095
:1025A2000C0E046E000E056E066E076E92EC09F0BC
:1025B20000C0F3F301C0F4F302C0F5F303C0F6F375
:1025C200050EF125E96E000EF221EA6E030EEE5CB5
:1025D200046E056A000E055A045000240401036FBC
:1025E20005500120046F000E05BEFF0E0220056F8C
:1025F200000E05BEFF0E0320066F03C4F3F304C4EE
:10260200F4F305C4F5F306C4F6F30C0E046E000EE3
:10261200056E066E076E03C400F004C401F005C423
:1026220002F006C403F0D8EC09F008C000F009C0BB
:1026320001F00AC002F00BC003F000C004F001C0B8
:1026420005F002C006F003C007F004360490053618
:1026520006360736070E04240301FF6F000E05201D
:102662000401006F000E0620016F000E0720026FAA
:102672006D0E006E010E016E000E026E036E03C43B
:1026820004F004C405F005C406F006C407F092EC99
:1026920009F00301FF5100260401005101220151FA
:1026A2000222025103220C0E046E000E056E066E0B
:1026B200076ED8EC09F000C0FFF301C000F402C0BD
:1026C20001F403C002F4FFC3F7F300C4F8F301C43A
:1026D200F9F302C4FAF3030E0301F125E96E000EC9
:1026E200F221EA6E300E046E000E056E066E076E63
:1026F20003C400F004C401F005C402F006C403F0F0
:10270200D8EC09F0EE500026000E0122022203222C
:10271200530E005E7D0E015A000E025A035A0050FB
:102722000301FF25046E015004010021056E0250D1
:102732000121066E03500221076E04C0F7F305C0A3
:10274200F8F306C0F9F307C0FAF3800E000A006E30
:10275200800E0718005C08E10650230805E10550C9
:10276200150802E1045023084FE2C00E046E120E57
:10277200056E000E066E076EF3C300F0F4C301F09F
:10278200F5C302F0F6C303F0D8EC09F000C0FFF382
:1027920001C000F402C001F403C002F4B00E046EE2
:1027A200040E056E000E066E076EF3C300F0F4C34E
:1027B20001F0F5C302F0F6C303F0D8EC09F0FFC351
:1027C20004F000C405F001C406F002C407F0005092
:1027D200045E0150055A0250065A0350075A260E4B
:1027E2000424006E000E0520016E000E0620026E0B
:1027F200000E0720036E00500301F7270150F82353
:102802000250F9230350FA230301040EF125FF6F4E
:10281200000EF2210401006F070E046E000E056E19
:10282200066E076EF7C300F0F8C301F0F9C302F0B9
:10283200FAC303F0D8EC09F008C000F009C001F0B7
:102842000AC002F00BC003F0FFC3E1FF00C4E2FFC5
:1028520000C0E6FF020E0301F125E96E000EF2212F
:10286200EA6EEECFFBF3000EFC6FFD6FFE6F000E03
:10287200FC6FFD6FFE6FFBC300F0FCC301F0FDC3F4
:1028820002F0FEC303F0100E046E0E0E056E000E73
:10289200066E000E076E92EC09F000C0FFF301C055
:1028A20000F402C001F403C002F4FFC3FBF300C44E
:1028B200FCF301C4FDF302C4FEF3010EF125E96E3F
:1028C200000EF221EA6EEECF00F0000E016E026EF3
:1028D200036E3C0E046E000E056E000E066E000EB8
:1028E200076E92EC09F00050FF25046E01500401BE
:1028F2000021056E02500121066E03500221076E6F
:1029020004C0FBF305C0FCF306C0FDF307C0FEF3F1
:10291200F1C3E9FFF2C3EAFFEECF00F00050042456
:102922000301FF6F000E05200401006F000E062058
:10293200016F000E0720026FFFC3FBF300C4FCF31C
:1029420001C4FDF302C4FEF3F7C300F0F8C301F0C3
:10295200F9C302F0FAC303F06250005E6350015AF9
:102962006450025A6550035A800E046E510E056E71
:10297200010E066E000E076E92EC09F00301FF5184
:1029820000260401005101220151022202510322B8
:02299200120031
:1029940002012B6B2C6B000E2C5D02E1800E2B5D73
:1029A40012E2680E2B25E16E030E2C21E26EE66A1C
:1029B400010E2B25006E000E2C21016E00C02BF29F
:1029C40001C02CF2E8D72B6B2C6B03014E6B4F6BC1
:1029D400AECF00F20201006B0301346B356B9D8AAC
:0829E400306B316BF28E120022
:1029EC007DEC2AF074EC0CF01A0E0B6E5E0E0C6E75
:1029FC006E0E0D6E0D2EFED70C2EFCD70B2EFAD7AD
:102A0C0000008B80080E0101A86F000EA96F899839
:102A1C00400EAF6EAC84C1EC0CF0030E0B6E8A0E44
:102A2C000C6E550E0D6E0D2EFED70C2EFCD70B2EEC
:102A3C00FAD7000000000C0E0401206FAEEC00F081
:102A4C000D0E0B6EAF0E0C6EB60E0D6E0D2EFED760
:102A5C000C2EFCD70B2EFAD70000040E0101A66F2A
:102A6C00010EA76F560E026F010E036F046B566BAF
:102A7C0056EC08F06F0E0401076F530E086F000E32
:102A8C00096F57EC09F00101546B556B800E551909
:102A9C00006E800E005C02E10A0E545D1CE2030E17
:102AAC00006E000E016E54C104F055C105F064ECCB
:102ABC0002F0320E0024E96E000E0120EA6EEECF19
:102ACC0007F4EECF08F4EECF09F457EC09F001014E
:102ADC00544B552BDBD7330E0B6EBB0E0C6EDF0E2F
:102AEC000D6E0D2EFED70C2EFCD70B2EFAD7000038
:102AFC00000056EC08F056EC08F0200E0101EE6FC9
:102B0C004E0EEF6FA6C1F1F3A7C1F2F33A0E03011B
:102B1C00F36F510EF46F000EF56F98EC0CF0EEC1E4
:102B2C00F1F3EFC1F2F3AE0E0301F36F010EF46F8C
:102B3C009FEC0BF0170E0101A6250301F16F000E9F
:102B4C000101A7210301F26FAE0EF36F010EF46FBA
:102B5C00050EF56F000EF66FF9EC0BF0A6C107F43D
:102B6C00A7C108F4F1EC08F05F0E076F510E086F67
:102B7C00000E096F57EC09F0040E0101A66F010E4F
:102B8C00A76F0301F16BF26BA6C1F3F3A7C1F4F3CA
:102B9C0021EC0CF056EC08F0820E0C6EDD0E0D6E76
:102BAC000D2EFED70C2EFCD700000000060E0101E6
:102BBC00A625E96E000EA721EA6E300EEE5C616E62
:102BCC000A0E6102F3CF61F0070EA625E96E000E26
:102BDC00A721EA6E300EEE5C006E00506126100EDE
:102BEC000301F16F000EF26FA6C1F3F3A7C1F4F36A
:102BFC0021EC0CF056EC08F0820E0C6EDD0E0D6E16
:102C0C000D2EFED70C2EFCD700000000040E010187
:102C1C00A625E96E000EA721EA6E300EEE5C606E02
:102C2C000A0E6002F3CF60F0050EA625E96E000EC9
:102C3C00A721EA6E300EEE5C006E00506026200E6E
:102C4C000301F16F000EF26FA6C1F3F3A7C1F4F309
:102C5C0021EC0CF056EC08F0820E0C6EDD0E0D6EB5
:102C6C000D2EFED70C2EFCD700000000060E010125
:102C7C00A625E16E000EA721E26EE66A040EA625DB
:102C8C000401076F000E0101A7210401086F86ECF7
:102C9C0008F000C0ABF1090E0101A625E16E000E93
:102CAC00A721E26EE66A070EA6250401076F000E47
:102CBC000101A7210401086F86EC08F000C0AAF1FD
:102CCC000101AD8160C05FF0300E0301F16F000EA9
:102CDC00F26FA6C1F3F3A7C1F4F321EC0CF056ECA0
:102CEC0008F0820E0C6EDD0E0D6E0D2EFED70C2E26
:102CFC00FCD700000000070E0101A625E96E000EAE
:102D0C00A721EA6E300EEE5C1D6E0A0E1D02F3CF8B
:102D1C001DF0080EA625E96E000EA721EA6E300EF6
:102D2C00EE5C006E00501D2656EC08F0230E0401DC
:102D3C00076F530E086F000E096F57EC09F0EAECA1
:102D4C000BF00001E66BE76B800E0301F16F0F0EC9
:102D5C00F26FF36B72EC0BF06AEC0CF0800EF16F0F
:102D6C000F0EF26FF36B330EF46F3CEC0BF06AEC5E
:102D7C000CF0800EF16F0F0EF26FF36BFFEC0AF09C
:102D8C0000C000F26AEC0CF0D50E0401076F530E74
:102D9C00086F000E096F57EC09F00101AE6B00C211
:102DAC00F1F3AE0E0301F26F010EF36FBFEC0AF0FC
:102DBC00AE0E0401076F010E086FF1EC08F0C80E9F
:102DCC00076F540E086F000E096F57EC09F00101E4
:102DDC00546B556B800E5519006E800E005C02E131
:102DEC00060E545D2AE2800E0301F16F0F0EF26F96
:102DFC00F36BFFEC0AF000C000F26AEC0CF0E80E8A
:102E0C0001015425E16E000E5521E26E00C2E6FF71
:102E1C00AE6B00C2F1F3AE0E0301F26F010EF36F55
:102E2C00BFEC0AF0AE0E0401076F010E086FF1EC57
:102E3C0008F00101544B552BCDD7B20E0401076F8E
:102E4C00540E086F000E096F57EC09F0800E030149
:102E5C00F16F0F0EF26FF36BFFEC0AF000C000F293
:102E6C000101AE6B00C2F1F3AE0E0301F26F010E65
:102E7C00F36FBFEC0AF0AE0E0401076F010E086F82
:102E8C00F1EC08F056EC08F0000E0401076F4F0E41
:102E9C00086F000E096F57EC09F0EDEC0CF051ECDB
:102EAC0011F0C70E076F520E086F000E096F57EC2A
:102EBC0009F0BBEC09F01A0E0B6E5E0E0C6E6E0E6A
:102ECC000D6E0D2EFED70C2EFCD70B2EFAD7000054
:102EDC000C0EC86ECCEC11F0C50E0401076F4E0E33
:102EEC00086F000E096F57EC09F081B246D0EFEC79
:102EFC0005F0EC0E0401076F500E086F000E096F01
:102F0C0057EC09F00401116B500E126F3AEC05F0FE
:102F1C00010E0401116F590E126F3AEC05F0170EE9
:102F2C000401076F61EC08F000C012F4020E116F7F
:102F3C003AEC05F0030E0401116F020E126F3AEC1D
:102F4C0005F0040E0401116F310E126F3AEC05F00E
:102F5C00050E0401116F120E126F3AEC05F0130EF0
:102F6C000401076F61EC08F000C012F4060E116F3B
:102F7C003AEC05F03DEC09F009D0A40E0401076F02
:102F8C00530E086F000E096F57EC09F056EC08F061
:102F9C0072EC06F0B50E0401076F530E086F000EAD
:102FAC00096F57EC09F0360E0401076F030E086F1A
:102FBC00F1EC08F0AA0E076F540E086F000E096FA3
:102FCC0057EC09F0440E0401076F030E086FF1EC87
:102FDC0008F056EC08F0F28CD08EF28CF28E080EC3
:102FEC000101A86F000EA96F56EC08F0BBEC09F0BC
:102FFC00970E076F500E086F000E096F57EC09F013
:10300C006D0E0301F16F540EF26F000EF36F140E80
:10301C00F46F000EF56FF2EC10F0880E0301F16FF7
:10302C00540EF26F000EF36F280EF46F000EF56F56
:10303C00F2EC10F089781A0E0B6E5E0E0C6E6E0EA2
:10304C000D6E0D2EFED70C2EFCD70B2EFAD70000D2
:10305C000101546B556B0A0E0401116F126B136B4B
:10306C00146B156B166B176B186B196B59EC05F011
:10307C001A0E0B6E5E0E0C6E6E0E0D6E0D2EFED7B6
:10308C000C2EFCD70B2EFAD700000F0E0101546F3B
:10309C00000E556F0A0E0401116F0F0E126F0F0EFA
:1030AC00136F0F0E146F0F0E156F0F0E166F0F0E92
:1030BC00176F0F0E186F0F0E196F59EC05F01A0ED3
:1030CC000B6E5E0E0C6E6E0E0D6E0D2EFED70C2E54
:1030DC00FCD70B2EFAD70000040E0101546F000E22
:1030EC00556F0A0E0401116F040E126F040E136F4C
:1030FC00040E146F040E156F040E166F040E176F6A
:10310C00050E186F050E196F59EC05F01A0E0B6EA3
:10311C005E0E0C6E6E0E0D6E0D2EFED70C2EFCD7A9
:10312C000B2EFAD70000BBEC09F0910E0301F16FE6
:10313C00540EF26F000EF36F61C0F4F3000EF56FD6
:10314C00F2EC10F0040E0101A66F010EA76FAC8B10
:10315C000001DD6B500E616EF29E51EC11F0BBEC78
:10316C0009F0760E0301F16F540EF26F000EF36F3F
:10317C0061C0F4F3000EF56FF2EC10F0BA0E04011E
:10318C00076F540E086F000E096F57EC09F0DDC085
:10319C00F1F3AE0E0301F26F010EF36F15EC11F0AB
:1031AC00AE0E0401076F010E086FF1EC08F056EC3F
:1031BC0008F0560E0101026F010E036F040EA66F8C
:1031CC00010EA76F72EC06F00001D56BD66BD76BB6
:1031DC00010ED86F010EDA6FD00E006E070E016E65
:1031EC001D500026D8B0012A00C0DBF001C0DCF075
:1031FC002DC2F1F30AEC12F000C0DEF02EC2F1F396
:10320C000AEC12F000C0DFF0EAC3F1F30AEC12F0A2
:10321C0000C0E0F0E8C3F1F30AEC12F000C0E1F0FA
:10322C00ECC3F1F30AEC12F000C0E3F0EBC3F1F3E2
:10323C000AEC12F0000E016ED00E0026070E0122D1
:10324C0000C0E4F001C0E5F0DE0EF16F000EF26F8D
:10325C00B9EC12F000C019F001C01AF002C01BF05A
:10326C0003C01CF0D50E0301F16F000EF26FB9EC28
:10327C0012F000C01EF001C01FF002C020F003C00D
:10328C0021F0D50E0301F16F000EF26FB9EC12F0C4
:10329C0000C0EDF301C0EEF302C0EFF303C0F0F396
:1032AC00DE0E0301F16F000EF26FB9EC12F0EDC3FC
:1032BC002CF0EEC32DF0EFC32EF0F0C32FF0005026
:1032CC002C5E01502D5A02502E5A03502F5A800E4C
:1032DC000301F16F0F0EF26FF36B72EC0BF0800EBB
:1032EC00F16F0F0EF26FF36BCC0EF46F3CEC0BF036
:1032FC00800EF16F0F0EF26FF36B440EF46F3CEC1B
:10330C000BF06AEC0CF0800EF16F0F0EF26FF36B9A
:10331C0072EC0BF0800EF16F0F0EF26FF36BCC0EA4
:10332C00F46F3CEC0BF0800EF16F0F0EF26FF36B41
:10333C00BE0EF46F3CEC0BF0800EF16F0F0EF26FC3
:10334C00F36BFFEC0AF000C02AF0000E2B6E800E1F
:10335C00F16F0F0EF26FF36BFFEC0AF000C031F05F
:10336C00306A2A5030262B503122CAEC14F080B629
:10337C00CFD0930E0401076F530E086F000E096F28
:10338C0057EC09F072EC06F0360E0401076F030ED1
:10339C00086FF1EC08F0200E206FAEEC00F0440E3C
:1033AC000401076F030E086FF1EC08F0200E206F7C
:1033BC00AEEC00F019C007F41AC008F41BC009F4F5
:1033CC001CC00AF4AE0E04010B6F010E0C6F03EC63
:1033DC0006F0AE0E076F010E086FF1EC08F056EC1C
:1033EC0008F0010E0401076F540E086F000E096FF0
:1033FC0057EC09F01EC0F1F31FC0F2F320C0F3F339
:10340C0021C0F4F3AE0E0301F56F010EF66F1FEC45
:10341C0012F0AE0E0401076F010E086FF1EC08F00C
:10342C0056EC08F0E40E0401076F530E086F000E03
:10343C00096F57EC09F02CC0F1F32DC0F2F32EC03C
:10344C00F3F32FC0F4F3F20E0301F56F000EF66FD9
:10345C001FEC12F0F20E0401076F000E086FF7EC70
:10346C0006F0F20E076F000E086FF1EC08F0270E55
:10347C00076F540E086F000E096F57EC09F02CC043
:10348C00F1F32DC0F2F3AE0E0301F36F010EF46FE6
:10349C009FEC0BF0AE0E0401076F010E086FF1EC00
:1034AC0008F0ED0E076F540E086F000E096F57EC05
:1034BC0009F0100E046E0E0E056E000E066E076EF1
:1034CC002CC000F02DC001F02EC002F02FC003F074
:1034DC00D8EC09F000C0F0F001C0F1F000C0F1F33D
:1034EC0001C0F2F3AE0E0301F36F010EF46F9FEC0B
:1034FC000BF0AE0E0401076F010E086FF1EC08F033
:10350C00510E076F540E086F000E096F57EC09F03F
:10351C001A0E0B6E5E0E0C6E6E0E0D6E0D2EFED711
:10352C000C2EFCD70B2EFAD70000800E2F18006E35
:10353C00800E005C08E1000E2E5C05E1000E2D5C97
:10354C0002E1040E2C5C42E27F0E006E800E2F18FE
:10355C00005C08E12E50FF0805E12D50FF0802E148
:10356C002C50880833E20F0E0101A86F000EA96FD2
:10357C0002C1F1F303C1F2F36A0E0301F36F500EB3
:10358C00F46F000EF56F98EC0CF002C107F403C158
:10359C0008F4F1EC08F056EC08F002C1F1F303C1A9
:1035AC00F2F361C0F3F3000E0301F46FA1EC12F01F
:1035BC000D0E0B6EAF0E0C6EB60E0D6E0D2EFED7E5
:1035CC000C2EFCD70B2EFAD7000053D1800E006EB8
:1035DC00800E2F18005C08E12E50000805E12D50DC
:1035EC00000802E12C50040851E2800E2F18006EE6
:1035FC00800E005C08E1000E2E5C05E1010E2D5CD6
:10360C0002E12C0E2C5C42E2190E616E0A0E0101D5
:10361C00A86F000EA96F560E026F010E036F02C148
:10362C00F1F303C1F2F3F60E0301F36F540EF46FD2
:10363C00000EF56F98EC0CF002C1F1F303C1F2F33C
:10364C00F20E0301F36F000EF46F30EC0EF002C1BA
:10365C00F1F303C1F2F3240EF36F000EF46F30ECB0
:10366C000EF002C1F1F303C1F2F3A6C1F3F3A7C14B
:10367C00F4F330EC0EF002C1F1F303C1F2F361C0CC
:10368C00F3F3000EF46FA1EC12F0F3D002C107F4C7
:10369C0003C108F475EC09F0800E026E800E01185F
:1036AC00025C02E1005007081CE20101ADA103D04D
:1036BC0060C05FF0AD915F5000080DE202C1F1F304
:1036CC0003C1F2F361C0F3F3000E0301F46FA1EC3C
:1036DC0012F05F0605D002C1E1FF03C1E2FFE66A0A
:1036EC00C8D00F0E0101A86F000EA96F040EA66FB3
:1036FC00010EA76FA6C1F1F3A7C1F2F3360E0301B9
:10370C00F36F030EF46F60EC0EF0A6C107F4A7C1C3
:10371C0008F475EC09F000C0F0F001C0F1F00050B5
:10372C000101A6250301F16F01500101A72103013D
:10373C00F26F220EF36F000EF46F30EC0EF0A6C198
:10374C0007F4A7C108F475EC09F000C0F0F001C053
:10375C00F1F000500101A6250301F16F01500101A8
:10376C00A7210301F26F440EF36F030EF46F30ECDC
:10377C000EF030C0F1F331C0F2F3AE0EF36F010E68
:10378C00F46FF4EC0CF0AE0E0401076F010E086F31
:10379C0075EC09F000C0F0F001C0F1F0AE0E0024A1
:1037AC000301F16F010E0120F26FF20EF36F540E54
:1037BC00F46F000EF56F98EC0CF0AE0E0401076F71
:1037CC00010E086FF1EC08F056EC08F0AE0E040197
:1037DC00076F010E086F75EC09F000C0F0F001C026
:1037EC00F1F00101546B556B800E5519006E800E73
:1037FC000001F119005C03E1F0510101545D15E287
:10380C000101AE0E5425E96E010E5521EA6EEE5003
:10381C00B00A08E1AE0E5425E16E010E5521E26EA0
:10382C007E0EE66E544B552BDFD7A6C107F4A7C10D
:10383C0008F475EC09F000C0F0F001C0F1F0005094
:10384C000101A6250301F16F01500101A72103011C
:10385C00F26FAE0EF36F010EF46F30EC0EF0A6C1EA
:10386C00F1F3A7C1F2F361C0F3F3000EF46FA1EC16
:10387C0012F00001DD2B816B300E0301445D006EF4
:10388C000A0E0002F3CF01F0300E455D006E0050C1
:10389C00012601C080F00101AA51015C06E3AB5185
:1038AC000001805D02E2010E816F0001000E805D5F
:1038BC0006E30101AA510001805DD8A0816B815102
:1038CC00000A0EE10A0E0401116F126B136B146BDC
:1038DC00156B166B176B186B196B59EC05F015D033
:1038EC0004010A0E116F020E126F020E136F020EFC
:1038FC00146F020E156F020E166F020E176F020E6A
:10390C00186F020E196F59EC05F0000E03013519F2
:10391C0002E1010E3419D8A41BEF23F0680EF16FED
:10392C00030EF26F9E0EF36F000EF46FECEC0DF0C5
:10393C0000C030F301C031F3000E026E0150025C86
:10394C0002E1005000083BE2680E0401076F030E11
:10395C00086F75EC09F000C0F0F001C0F1F0800EBA
:10396C00026E800E0118025C02E1005006081FE294
:10397C00800E0001F119006E800E005C02E1540E05
:10398C00F05D15E2820E0401076F000E086FF1EC7A
:10399C0008F002C1F1F303C1F2F36C0E0301F36FF3
:1039AC00030EF46F60EC0EF00101AD8105D002C185
:1039BC00E1FF03C1E2FFE66A0301306B316B0301E7
:1039CC00680EF16F030EF26F710EF36F000EF46F51
:1039DC00ECEC0DF000C030F301C031F3000E026EC0
:1039EC000150025C02E10050000818E20101AC8BAE
:1039FC00680E0401076F030E086F75EC09F000C028
:103A0C00F0F001C0F1F0F60E076F520E086F000EC9
:103A1C00096F57EC09F00301306B316B0301680E31
:103A2C00F16F030EF26F680EF36F000EF46FECEC97
:103A3C000DF000C030F301C031F3000E026E0150E6
:103A4C00025C02E1005000080EE20101AC9B3A0E50
:103A5C000401076F500E086F000E096F57EC09F048
:103A6C000301306B316B0301680EF16F030EF26FC3
:103A7C00790EF36F000EF46FECEC0DF000C030F328
:103A8C0001C031F3000E026E0150025C02E10050E5
:103A9C000008D8B0E0D00201276B286B060E03019A
:103AAC003025E96E000E3121EA6EEECF11F458ECA0
:103ABC0002F00052D8B4C3D0070E03013025E96ED2
:103ACC00000E3121EA6EEECF11F458EC02F00052E8
:103ADC00D8B4B5D0060E03013025E96E000E3121A5
:103AEC00EA6E300EEE5C006E016A000E015A0A0E90
:103AFC00046E000E056E64EC02F000C0EDF301C024
:103B0C00EEF3EDC327F2EEC328F2070E3025E96E73
:103B1C00000E3121EA6E300EEE5C006E016A000E72
:103B2C00015A0A0E046E000E056E87EC0EF008C0EA
:103B3C0000F009C001F000500301ED25026E0150A8
:103B4C00EE21036E02C027F203C028F2800E006E35
:103B5C00800E0318005C02E10250090866E2800E38
:103B6C0002012819006E800E005C02E1640E275DD4
:103B7C005CE2F30E0401076F530E086F000E096F21
:103B8C0057EC09F061C0F1F3AE0E0301F26F010EB8
:103B9C00F36F15EC11F0AE0E0401076F010E086FF8
:103BAC00F1EC08F056EC08F027C261F0060E0301A8
:103BBC00F16F060E3025E96E000E3121EA6EEECF64
:103BCC00F2F35AEC10F0A30E0C6E550E0D6E0D2E7A
:103BDC00FED70C2EFCD7070E0301F16F070E302514
:103BEC00E96E000E3121EA6EEECFF2F35AEC10F0D2
:103BFC00A30E0C6E550E0D6E0D2EFED70C2EFCD793
:103C0C00E10E0401076F540E086F000E096F57EC9C
:103C1C0009F00301F16BF26BAE0EF36F010EF46F52
:103C2C0021EC0CF056EC08F009D0840E0401076F5F
:103C3C00510E086F000E096F57EC09F009D0CA0E2F
:103C4C000401076F510E086F000E096F57EC09F055
:103C5C000301306B316B0301680EF16F030EF26FD1
:103C6C00A30EF36F000EF46FECEC0DF000C030F30C
:103C7C0001C031F3000E026E0150025C02E10050F3
:103C8C000008D8B0E2D00201276B286B040E0301A8
:103C9C003025E96E000E3121EA6EEECF11F458ECAE
:103CAC0002F00052D8B4C5D0050E03013025E96EE0
:103CBC00000E3121EA6EEECF11F458EC02F00052F6
:103CCC00D8B4B7D0040E03013025E96E000E3121B3
:103CDC00EA6E300EEE5C006E016A000E015A0A0E9E
:103CEC00046E000E056E64EC02F000C0EDF301C032
:103CFC00EEF3EDC327F2EEC328F2050E3025E96E84
:103D0C00000E3121EA6E300EEE5C006E016A000E80
:103D1C00015A0A0E046E000E056E87EC0EF008C0F8
:103D2C0000F009C001F000500301ED25026E0150B6
:103D3C00EE21036E02C027F203C028F2800E006E43
:103D4C00800E0318005C02E10250000868E2800E4D
:103D5C0002012819006E800E005C02E10B0E275D3B
:103D6C005EE21B0E0401076F540E086F000E096F04
:103D7C0057EC09F060C0F1F3AE0E0301F26F010EC7
:103D8C00F36F15EC11F0AE0E0401076F010E086F06
:103D9C00F1EC08F056EC08F027C260F0140E0301A9
:103DAC00F16F040E3025E96E000E3121EA6EEECF74
:103DBC00F2F35AEC10F0A30E0C6E550E0D6E0D2E88
:103DCC00FED70C2EFCD7150E0301F16F050E302516
:103DDC00E96E000E3121EA6EEECFF2F35AEC10F0E0
:103DEC00A30E0C6E550E0D6E0D2EFED70C2EFCD7A1
:103DFC00E70E0401076F540E086F000E096F57ECA5
:103E0C0009F0100E0301F16F000EF26FAE0EF36F9E
:103E1C00010EF46F21EC0CF056EC08F009D0A80E52
:103E2C000401076F510E086F000E096F57EC09F073
:103E3C0009D02E0E0401076F520E086F000E096F89
:103E4C0057EC09F00301306B316B0301680EF16F15
:103E5C00030EF26FBE0EF36F000EF46FECEC0DF070
:103E6C0000C030F301C031F3000E026E0150025C51
:103E7C0002E100500008D8B07BD00201276B286B00
:103E8C00070E03013025E96E000E3121EA6EEECFEC
:103E9C0011F458EC02F0005268E0070E03013025D3
:103EAC00E96E000E3121EA6E300EEE5C016E026A94
:103EBC00000E025A01C027F202C028F2800E006EDA
:103ECC00800E0218005C02E10150000845E2800EF1
:103EDC0002012819006E800E005C02E1070E275DBE
:103EEC003BE2050E006E27C2F0F028C2F1F0005044
:103EFC0006E00001F037F091F137FF0FF9D7000120
:103F0C00200EF027000EF1230D0E0401076F530E47
:103F1C00086F000E096F57EC09F0F0C0F1F3F1C017
:103F2C00F2F3AE0E0301F36F010EF46F79EC10F0A7
:103F3C00AE0E0401076F010E086FF1EC08F056ECA1
:103F4C0008F002C1F1F303C1F2F3F0C0F3F3F1C0D6
:103F5C00F4F3EBEC0EF009D0090E0401076F500ED0
:103F6C00086F000E096F57EC09F00301306B316BD1
:103F7C0003016851550A2AE17B51230A27E130ECF1
:103F8C000FF0810E0401076F530E086F000E096FBE
:103F9C0057EC09F0360E0401076F030E086FF1ECB5
:103FAC0008F00F0E076F540E086F000E096F57ECD8
:103FBC0009F0440E0401076F030E086FF1EC08F0D2
:103FCC0056EC08F00301686B306B316B680EF16FC7
:103FDC00030EF26FB90EF36F000EF46FECEC0DF0F4
:103FEC0000C030F301C031F3000E026E0150025CD0
:103FFC0002E10050000878E27A0E0401076F4D0EC2
:10400C00086F000E096F57EC09F0010E0101546F97
:10401C00000E556F800E5519006E800E005C02E18B
:10402C00050E545D5EE2050E026E54C100F055C1E2
:10403C0001F0025005E0003600900136FF0FFAD770
:10404C0000C0F0F001C0F1F0A6C1F1F3A7C1F2F38A
:10405C0000C0F3F301C0F4F3EBEC0EF0470E0401D7
:10406C00076F540E086F000E096F57EC09F0F0C083
:10407C00F1F3F1C0F2F3AE0E0301F36F010EF46F26
:10408C0079EC10F0AE0E0401076F010E086FF1EC25
:10409C0008F0090E206FAEEC00F0A6C107F4A7C122
:1040AC0008F4F1EC08F056EC08F0A6C1F1F3A7C146
:1040BC00F2F361C0F3F3000E0301F46FA1EC12F004
:1040CC001A0E0B6E5E0E0C6E6E0E0D6E0D2EFED756
:1040DC000C2EFCD70B2EFAD700000101544B552B9C
:1040EC0099D70301306B316B0301680EF16F030E2E
:1040FC00F26FCB0EF36F000EF46FECEC0DF000C012
:10410C0030F301C031F3000E026E0150025C02E18B
:10411C000050000825E24E0E0401076F520E086F86
:10412C00000E096F57EC09F051EC11F0DF0E076F20
:10413C00520E086F000E096F57EC09F0BBEC09F03A
:10414C001A0E0B6E5E0E0C6E6E0E0D6E0D2EFED7D5
:10415C000C2EFCD70B2EFAD700000301306B316B01
:10416C000301680EF16F030EF26FC60EF36F000EB3
:10417C00F46FECEC0DF000C030F301C031F3000E25
:10418C00026E0150025C02E1005000080EE23C0E8F
:10419C000401076F4A0E086F000E096F57EC09F007
:1041AC0056EC08F00301306B316B0301680EF16FB4
:1041BC00030EF26FA80EF36F000EF46FECEC0DF023
:1041CC0000C030F301C031F3000E026E0150025CEE
:1041DC0002E100500008D8B0AFD0680E0401076FA0
:1041EC00030E086F75EC09F0000E011802E1090EC0
:1041FC000018D8A4A1D0320E076F540E086F000E11
:10420C00096F57EC09F0300E0301F16F000EF26FDD
:10421C00A6C1F3F3A7C1F4F321EC0CF056EC08F0B3
:10422C00820E0C6EDD0E0D6E0D2EFED70C2EFCD7F5
:10423C0000000000070E03013025E96E000E31214D
:10424C00EA6EEECF11F458EC02F000C0EDF3080E5C
:10425C0003013025E96E000E3121EA6EEECF11F428
:10426C0058EC02F000500301ED25016E026A000EBD
:10427C00022201C029F202C02AF2800E006E800ECA
:10428C000218005C02E1015014084AE2800E02019F
:10429C002A19006E800E005C02E1630E295D40E27B
:1042AC00070E03013025E96E000E3121EA6EEECFC8
:1042BC0000F2370EF16F00C2F2F35AEC10F0820EDE
:1042CC000C6EDD0E0D6E0D2EFED70C2EFCD70000E5
:1042DC000000300E0201005D1D6E0A0E1D02F3CFB0
:1042EC001DF0080E03013025E96E000E3121EA6E37
:1042FC00EECF00F2380EF16F00C2F2F35AEC10F070
:10430C00820E0C6EDD0E0D6E0D2EFED70C2EFCD714
:10431C0000000000020100511D26300E1D5E09D068
:10432C00D70E0401076F4F0E086F000E096F57EC84
:10433C0009F00301306B316B0301680EF16F030E52
:10434C00F26FB40EF36F000EF46FECEC0DF000C0D6
:10435C0030F301C031F3000E026E0150025C02E139
:10436C0000500008D8B05ED1680E0401076F030E30
:10437C00086F75EC09F0800E0118026E800E025C5D
:10438C0002E1090E005CD8A04DD1090E03013025C5
:10439C00E16E000E3121E26EE66AA20E0401076F97
:1043AC00540E086F000E096F57EC09F0200E030134
:1043BC00F16F000EF26FAE0EF36F010EF46F21EC85
:1043CC000CF0040E3025E96E000E3121EA6EEECFB2
:1043DC0011F458EC02F000C0EDF3050E030130258A
:1043EC00E96E000E3121EA6EEECF11F458EC02F0BA
:1043FC0000500301ED27EE6B000EEE23070E302567
:10440C00E96E000E3121EA6EEECF11F458EC02F099
:10441C0000500301ED27000EEE23080E3025E96E47
:10442C00000E3121EA6EEECF11F458EC02F0005080
:10443C000301ED27000EEE23EDC329F2EEC32AF2A1
:10444C00040E3025E96E000E3121EA6E300EEE5C62
:10445C00006E016A000E015A0A0E046E000E056E03
:10446C0064EC02F0050E3025D96E000E3121DA6EA7
:10447C00DE5000240001F06F000E0120F16F300EB1
:10448C00F05F000EF15B070E03013025E96E000EA4
:10449C003121EA6E300EEE5C006E016A000E015A9C
:1044AC000A0E046E000E056E64EC02F0080E302548
:1044BC00D96E000E3121DA6EDE5000240201276F16
:1044CC00000E0120286F300E275F000E285B000EB7
:1044DC000301EE1902E1040EED19D8A495D0800E5B
:1044EC000001F119006E800E005C02E10F0EF05D10
:1044FC00D8A08AD0800EF119006E800E005C02E10B
:10450C00180EF05DD8B080D0800E006E800E0201C7
:10451C002819005C02E12751030876E2800E006E38
:10452C00800E2819005C02E127510B086DE3F0C0E6
:10453C00ABF1040E03013025E96E000E3121EA6E59
:10454C00EECF00F2240EF16F00C2F2F35AEC10F031
:10455C00050E03013025E96E000E3121EA6EEECF17
:10456C0000F2250EF16F00C2F2F35AEC10F0A30E1C
:10457C000C6E550E0D6E0D2EFED70C2EFCD727C2D1
:10458C00AAF1070E03013025E96E000E3121EA6E07
:10459C00EECF00F2270EF16F00C2F2F35AEC10F0DE
:1045AC00A30E0C6E550E0D6E0D2EFED70C2EFCD7D9
:1045BC00080E03013025E96E000E3121EA6EEECFB4
:1045CC0000F2280EF16F00C2F2F35AEC10F0A30EB9
:1045DC000C6E550E0D6E0D2EFED70C2EFCD79A0EB2
:1045EC000401076F540E086F000E096F57EC09F0A9
:1045FC00200E0301F16F000EF26FAE0EF36F010E81
:10460C00F46F21EC0CF009D0380E0401076F4F0E3B
:10461C00086F000E096F57EC09F056EC08F0030117
:10462C00306B316B0301306B316BB2EF18F0FFD78D
:1054FA0010EE19F0BC0E006E010E016E270EF66E4C
:0E550A004C0EF76E000EF86E62EC0CF0120004
:10463C00000000000000000000000000000000006E
:10464C00000000000000000000000000000000005E
:10465C00000000000000000000000000000000004E
:10466C00000000000000000000000000000000003E
:10467C00000000000000000000000000000000002E
:10468C00000000000000000000000000000000001E
:10469C00000000000000000000000000000000000E
:1046AC0000000000000000000000000000000000FE
:1046BC0000000000000000000000000000000000EE
:1046CC0000000000000000000000000000000000DE
:1046DC0000000000000000000000000000000000CE
:1046EC0000000000000000000000000000000000BE
:1046FC0000000000000000000000000000000000AE
:10470C00000000000000000000000000000000009D
:10471C00000000000000000000000000000000008D
:10472C00000000000000000000000000000000007D
:10473C00000000000000000000005F00000000000E
:10474C000007000700000000147F147F1400000015
:10475C00242A7F2A1200000026160834320000009A
:10476C0076495522500000000000050300000000AF
:10477C00001C2241000000000041221C000000002F
:10478C0014083E081400000008083E080800000049
:10479C000050300000000000080808080800000065
:1047AC0000606000000000002010080402000000FF
:1047BC003E5149453E00000000427F400000000091
:1047CC0042615149460000002141454B3100000037
:1047DC001814127F100000002745454539000000D1
:1047EC003C4A4949300000000101790503000000F2
:1047FC003649494936000000064949291E00000087
:10480C0000363600000000000056360000000000A4
:10481C0000081422410000001414141414000000A9
:10482C00412214080000000002015109060000009A
:10483C003E4149555E0000007E1111117E000000C2
:10484C007F494949360000003E41414122000000A9
:10485C007F4141221C0000007F4949494100000072
:10486C007F090909010000003E4149493A00000056
:10487C007F0808087F00000000417F410000000015
:10488C002041413F000000007F081422410000003D
:10489C007F404040400000007F020C027F0000007F
:1048AC007F0408107F0000003E4141413E000000A3
:1048BC007F090909060000003E4151215E000000FD
:1048CC007F0919294600000046494949310000007A
:1048DC0001017F01010000003F4040403F0000000B
:1048EC001F2040201F0000003F403C403F000000C4
:1048FC006314081463000000070870080700000028
:10490C006151494543000000007F41410000000017
:10491C0002040810200000000041417F000000004C
:10492C00040201020400000040404040400000002E
:10493C0000010204000000002054545478000000D0
:10494C007F484444380000003844444420000000B0
:10495C00384444487F000000385454541800000078
:10496C00087E090102000000085454543C00000069
:10497C007F0804047800000000447D400000000023
:10498C002040443D000000007F102844000000003F
:10499C0000417F40000000007C04180478000000F7
:1049AC007C080404780000003844444438000000BB
:1049BC007C14141408000000081414187C00000067
:1049CC007C080404080000004854545420000000E3
:1049DC00043F4440200000003C4040207C0000008C
:1049EC001C2040201C0000003C4038403C000000D3
:1049FC0044281028440000000C5050503C0000008B
:104A0C004464544C4400000000083641000000008F
:104A1C0000007F000000000000413608000000008C
:104A2C000000060909060000001038541010100090
:104A3C003C4D73673D3E2020204C206D6178693DD4
:104A4C0031323020636172730D0A3C5265736574A8
:104A5C003E202052652D496E69742061666669633B
:104A6C006865757273204D4158373231390D0A3CE7
:104A7C0054454D505F4F4E3E202020416666696381
:104A8C006865206C612054656D702E20445331385C
:104A9C004232300D0A3C54454D505F4F46463E2045
:104AAC0020456E6C65766520416666696368616752
:104ABC006520445331384232300D0A3C53706565E1
:104ACC00643D33303E202020566974657373652035
:104ADC00646566696C656D656E74203A76616C65AB
:104AEC00757220646520313020E02039390D0A3C84
:104AFC00456570726F6D3D323E2020204D6573739D
:104B0C0061676520656E20656570726F6D206465E8
:104B1C002033322063617273202C617665632069C7
:104B2C006E64696365203120E020360D0A3C504CE0
:104B3C004D3D31383A30363E20506C616765204C23
:104B4C00756D696E6F736974E9204D696E696D617D
:104B5C006C65200D0A3C5265703D30313E202020A2
:104B6C0052657065746974696F6E204D65737361FD
:104B7C0067652020303120E02031300D0A3C416E39
:104B8C004E6575663D32313E204E6F7576656C20F4
:104B9C00414E203D20323030302B20416E4E657519
:104BAC006620323120E02039380D0A3C553B303438
:104BBC003B30363B31393B32303B35393B3034239B
:104BCC003E20204D616A206465206C612052544364
:104BDC0020553B4A4A3B4D4D3B41413B48483B4DA0
:104BEC004D3B4A5323200D0A3C44656D6F3E2020FB
:104BFC00206166666963686520746F7573206C65E7
:104C0C0073206D6573736167657320656E20454510
:0B4C1C0050524F4D205049430D0A003C
:044C27000000000089
:014C2B001474
:044C2C000000000084
:024C3000200062
:064C320020536563200021
:024C380000007A
:044C3A000000000076
:024C3E00000074
:104C4000C250002F4D00864E00BF4D00145100E3AE
:104C50004C004A5300AC5200034E00A44F00A44F36
:0D4C6000006E5200375300EC51005B540011
:014C6D000046
:014C6E000441
:014C6F001E26
:044C70008C3D250052
:024C740000003E
:094C760054454D505F4F464600C5
:084C7F0054454D505F4F4E00FB
:074C870053706565643D00F8
:014C8E000025
:014C8F000024
:104C90000D0A2068656C6C6F2C2069206765742094
:0C4CA000796F7572204D7367210D0A00BA
:054CAC004D73673D009F
:054CB1005265703D009A
:084CB600416E4E6575663D007C
:044CBE0000000000F2
:054CC200504C4D3D00C7
:054CC70044656D6F0063
:084CCC00456570726F6D3D003B
:054CD40048656C700052
:064CD900526573657400D2
:044CDF0000000000D1
:104CE300205350493120536F667477202D3E204D59
:104CF3004158373231392C2049324331204857202B
:104D03002D3E204453313330372C205541525431FA
:104D130020313930302C382C4E2C312C204F575326
:0C4D23002D3E445331384232300D0A005E
:104D2F00204469726563746F7279203A20433A5C4C
:104D3F005F4D696B726F435C5F4D657350726F6A45
:104D4F006574735F4D696B726F430138463235324C
:104D5F005F4D73675F446566696C5F385F4D617463
:0B4D6F0072696365735F56200D0A0037
:104D7A00416666696368652036204D6573736167AD
:104D8A00657320656E20454550524F4D206D6F6406
:104D9A00756C6F20333220E0207061727469722062
:104DAA006465203078303034302E2E3078303045FB
:054DBA0030200D0A008D
:104DBF0020536F75726365203A204D657373616779
:104DCF00655F446566696C616E745F38784D6178B4
:104DDF00373231395F4D617472696365735F565F46
:104DEF003138463235325F323032305F30312E63F8
:044DFF00200D0A0079
:104E03002038204D617472696365732038783820C7
:104E1300726163636F7264656D656E74207665722B
:104E2300746963616C204841555420766572732020
:104E330042617320737572204D4158373132390DF9
:024E43000A0063
:104E450020553A30333B31323B31393B31383B33F6
:104E5500363B3032232020706F757220303320644A
:104E65006563656D627265203230313920203138D5
:104E75004833362030323D4D617264690D0A0D0AA2
:014E8500002C
:104E86002050726F6A6574203A204D6573736167AE
:104E9600655F446566696C616E745F38784D6178EC
:104EA600373231395F4D617472696365735F565F7E
:0F4EB6003138463235322E6D637070690D0A0047
:104EC500496E6974204932433220285243333D5399
:104ED500434C206574205243343D534441202934CA
:104EE50030304B687A200D0A20496E69742052547F
:0B4EF50043204453313330370D0A00D6
:104F0000496E69742053504920536F6674776172FB
:104F1000652020524332202853434B292C205243F2
:104F200031202853444F2C292065742052433020CF
:084F300028435329200D0A005B
:104F38002042414420504C4D2076616C75657321A8
:104F4800206D7573742062652066726F6D205B3109
:104F5800352E2E203233205D20746F205B203420C4
:084F68002E2E203131205D00E6
:104F70000D0A2052617070656C20666F726D6174ED
:104F800020646520636465203A2022553B4A4A3BF1
:104F90004D4D3B41413B48483B4D4D3B6A442322EC
:044FA000200D0A00D6
:104FA4002053616973697220756E206E6F75766522
:104FB4006175204D73672061766563206C6520748C
:104FC40065726D696E616C20766961204D73673D11
:034FD4000D0A00C3
:104FD7002042414420416E4E6575662076616C75AE
:104FE700652021206D75737420626520696E2074B9
:104FF70068652072616E6765203231202E2E203958
:0250070038006F
:105009000D0A20456570726F6D204D7367206164CC
:10501900726573736520206D7573742062652077DE
:10502900697468696E203120746F20373E3E0D0A1D
:015039000076
:10503A000D0A204F4B2C2054656D706572206973E0
:10504A00204F4646210D0A5265746F7572206175AC
:10505A0020646973706C617920747874200D0A0079
:10506A0020426F6E6E6520416E6E65652032303269
:10507A003120657420426F6E6E652053616E7465CF
:0D508A0020426967204269736F7573200032
:1050970020446973706C6179203C30313233343588
:1050A70036373E207375722038206D6174726963DC
:0B50B7006573204C656473200D0A0037
:1050C200204C616E6761676520204D696B726F636A
:1050D200205620372E36300D0A204D4355203A20D7
:0A50E200313846323532200D0A0045
:1050EC00696E697420525443207061722064656645
:1050FC006175742033312F31322F323031392032F7
:08510C00333A35393A30300026
:1051140020436F6E6669672042697473205031388A
:10512400463235325F515F31304D487A2E636667BF
:065134007363680D0A0020
:10513A000D0A20436C6F636B20696E697469616C38
:10514A006520696E20203D20202E2E2E20204B68BF
:05515A007A200D0A009F
:10515F0020526563757020506172616D6574726560
:10516F007320656E2045656570726F6D20504943E1
:05517F00203A0D0A00BA
:105184000D0A205370656564206D75737420626523
:105194002077697468696E20313020746F20393942
:0451A400200D0A00D0
:1051A8000D0A20526570206D757374206265207732
:1051B800697468696E20303120746F203130200D99
:0251C8000A00DB
:1051CA000D0A2042414420636465202C206D7573CA
:1051DA00742062653A2053706565643D7878200DC5
:0251EA000A00B9
:1051EC0020426F6E6E6520416E6E656520323032E6
:1051FC0031202C20424F4E4E452053414E544520D9
:01520C0000A1
:10520D000D0A45727265757220737572204A6F753D
:10521D00722053656D61696E65206A532E200D0AEB
:01522D000080
:10522E000D0A2042414420636465202C206D757365
:10523E00742062653A205265703D7878200D0A0020
:10524E00526573657420416666696368657572732D
:10525E00204D61747269636520387838200D0A001C
:10526E00204D6F64652054656D7065726174757242
:0F527E006520617665632054454D505F4F4E00AB
:10528D000D0A45637269747572652064616E7320D1
:0F529D004453313330372E2E2E204F4B0D0A0045
:1052AC0020454550524F4D203A2E2E2E5F454550ED
:0B52BC00524F4D2E696865780D0A0006
:1052C70020436C656172204D617472696365203893
:0852D70078203878380D0A0038
:1052DF00436C656172204D61747269636520367825
:0752EF00203878380D0A0099
:1052F6000D0A204F4B2C2054656D70657220697322
:07530600204F4E210D0A00AB
:10530D002020456570726F6D204D7367206164724A
:06531D00657373652000BA
:1053230054657374207265672E20445331384232BA
:04533300300D0A002F
:10533700204A6F79657578204E4F454C20323032C0
:0353470030200013
:10534A0020506F77657220537570706C79203556CE
:03535A000D0A0039
:10535D000A0D205254432055704461746564200D2C
:02536D000A0034
:10536F002050726573656E746174696F6E203A0DAB
:02537F000A0022
:105381004E657720445331333037204461746520B2
:025391003A00E0
:10539300204461746520267431204E6F77203D20B0
:0153A3000009
:1053A4002052652D4C6563747572652052544320F8
:0153B40000F8
:1053B500204453313330372044617465203A20004E
:1053C5003031323334353637383941424344454636
:0F53D50046616D696C7920436F6465203A200052
:0F53E40020446966666572656E6365203D200032
:0E53F300204F6C64207370656564203D2000BF
:0E54010020446174652026543220203D200096
:0C540F00204E65772054696D653A20003E
:0C541B00204F6C6420526570203D200082
:0B5427002020736F6974203D3E2000C0
:0B54320020416E4E657566203D200095
:0A543D004D657263726564692E000C
:0A544700456570726F6D2023200090
:0A545100204865757265730D0A00AE
:09545B0020787878787878200038
:0954640056656E6472656469000E
:09546D0020202020202020200036
:095476002020202020202020002D
:09547F0044696D616E636865000B
:095488003031323334353637007F
:0954910020202020202020200012
:08549A00204E6577203D200043
:0854A200204F6C64203D200046
:0854AA002054696D653A2000F1
:0854B20020204352433D20007D
:0754BA00204370743D200047
:0754C10053616D6564690091
:0754C800204944313D2000A2
:0654CF004C756E646900DB
:0654D5004D6172646900E4
:0654DB004A6575646900DA
:0654E100204E657720005B
:0654E700204E6577200055
:0554ED00202D3E20000F
:0454F200B0432000A3
:0454F6003E3E200016
:020000040030CA
:0D000100220F0EFF0181FF0FC00FE00F4026
:0200000400F00A
:1000000053706565643D333000FFFFFFFFFFFFFF66
:100010005265703D303400FFFFFFFFFFFFFFFFFF21
:10002000504C4D3D31393A303500FFFFFFFFFFFFA7
:10003000416E4E6575663D323100FFFFFFFFFFFFE9
:10004000504943313846323532204D696B726F4327
:100050005665722E50726F20562E372E363000FFA6
:1000600032656D20436F75636F752000FFFFFFFFE2
:10007000FFFFFFFFFFFFFFFFFFFFFFFFFFFFFFFF90
:1000800033656D20204F756920204F4B204241443D
:1000900000FFFFFFFFFFFFFFFFFFFFFFFFFFFFFF6F
:1000A00034656D206D6573736167652020202020A5
:1000B0002020202020202020202020202020200060
:1000C00035656D204D73672E2E2E2E2E2E2E2E2E44
:1000D0002E2E2E2E2E2E2E2E2E2E2E2E2E2E2E006E
:1000E00036656D204D657373616765202020202083
:1000F0002E2E2E2E2E2E2E2E2E2E2E2E2E2E2E004E
:00000001FF
